:020000040800F2
:1000000000A0002099080008C9060008D7060008CB
:10001000DD060008E3060008E9060008000000000D
:10002000000000000000000000000000EF060008D3
:10003000FD060008000000000B0700081907000873
:10004000E9080008E9080008E9080008E9080008CC
:10005000E9080008E9080008E9080008E9080008BC
:10006000E9080008E9080008E9080008E9080008AC
:10007000E9080008E9080008E9080008E90800089C
:10008000E9080008E9080008E90800080000000085
:10009000000000000000000000000000E908000867
:1000A000E9080008E9080008E9080008E90800086C
:1000B000E90800080000000000000000E90800084E
:1000C000E9080008E9080008E9080008E90800084C
:1000D000E9080008E9080008E9080008E90800083C
:1000E000E9080008E908000800000000000000001E
:1000F0000000000000000000000000000000000000
:1001000000000000000000000000000000000000EF
:100110000000000000000000E908000800000000E6
:10012000E9080008E9080008E9080008E9080008EB
:10013000E9080008000000000000000000000000C6
:10014000E9080008E9080008E908000800000000C4
:10015000E9080008E9080008E9080008E9080008BB
:10016000E9080008E908000800000000000000009D
:1001700000000000E9080008000000000000000086
:0C018000E9080008E9080008E908000888
:10018C0010B5054C237833B9044B13B10448AFF3C5
:10019C0000800123237010BD0C0000200000000023
:1001AC002029000808B5034B1BB103490348AFF3E2
:1001BC00008008BD0000000010000020202900086D
:1001CC0053B94AB9002908BF00281CBF4FF0FF31B2
:1001DC004FF0FF3000F072B9ADF1080C6DE904CEB0
:1001EC0000F006F8DDF804E0DDE9022304B0704706
:1001FC002DE9F047089E04468846002B4BD18A42D5
:10020C00154667D9B2FA82F24AB1C2F1200701FA57
:10021C0002F320FA07F7954047EA030894404FEAA7
:10022C00154E230CB8FBFEF71FFA85FC0EFB178846
:10023C0043EA084307FB0CF1994209D9EB1807F183
:10024C00FF3080F01B81994240F21881023F2B4411
:10025C005B1AA4B2B3FBFEF00EFB103344EA03446A
:10026C0000FB0CFCA44509D92C1900F1FF3380F0DC
:10027C000781A44540F2048102382C4440EA07402F
:10028C00A4EB0C0400271EB1D4400023C6E90043A4
:10029C003946BDE8F0878B4209D9002E00F0EB807F
:1002AC000027C6E9000138463946BDE8F087B3FAA5
:1002BC0083F7002F47D18B4202D3824200F2FA809F
:1002CC00841A61EB030301209846002EE0D0C6E9A6
:1002DC000048DDE702B9FFDEB2FA82F2002A40F0F4
:1002EC008F80491B4FEA154E1FFA85F80127B1FB89
:1002FC00FEFC230C0EFB1C1143EA014308FB0CF122
:10030C00994207D9EB180CF1FF3002D2994200F256
:10031C00CD808446591AA3B2B1FBFEF00EFB10142B
:10032C0043EA044408FB00F8A04507D92C1900F156
:10033C00FF3302D2A04500F2B6801846A4EB0804A5
:10034C0040EA0C409FE7C7F1200CBB4022FA0CFEA0
:10035C004EEA030E01FA07F420FA0CF521FA0CF31D
:10036C004FEA1E482543B3FBF8F92C0C08FB193354
:10037C001FFA8EFA44EA034309FB0AF49C4202FA80
:10038C0007F200FA07F10BD91EEB030309F1FF305A
:10039C0080F087809C4240F28480A9F1020973446A
:1003AC001B1BADB2B3FBF8F008FB103345EA03445A
:1003BC0000FB0AFAA24508D91EEB040400F1FF3336
:1003CC006BD2A24569D90238744440EA0940A0FBBB
:1003DC000289A4EB0A044C45C2464B4654D351D077
:1003EC00002E69D0B1EB0A0564EB030404FA0CFC93
:1003FC00FD40FC404CEA0505C6E90054002747E7E0
:10040C00C2F1200320FA03F7954001FA02F021FA19
:10041C0003F34FEA154E3843010CB3FBFEF71FFAFA
:10042C0085F80EFB173341EA034107FB08F38B42B7
:10043C0004FA02F407D9691807F1FF3C2FD28B425A
:10044C002DD9023F2944CB1A81B2B3FBFEF00EFB2F
:10045C00103341EA034100FB08F38B4207D96918BA
:10046C0000F1FF3C17D28B4215D902382944C91A26
:10047C0040EA07473BE73746304609E70746E7E6D9
:10048C001846FBE64145ABD2B8EB020A69EB0E020B
:10049C0001381346A4E76046E9E7184695E7674636
:1004AC00D1E781467CE702382C4447E7ACF1020CDB
:1004BC002B442FE7384608E73746E9E6704700BF7C
:1004CC0080B588B000AF07F10C0300221A605A60A7
:1004DC009A60DA601A61264BDB6C254A43F0040300
:1004EC00D364234BDB6C03F00403BB60BB68204B71
:1004FC00DB6C1F4A43F00103D3641D4BDB6C03F030
:10050C0001037B607B681A4BDB6C194A43F00203D6
:10051C00D364174BDB6C03F002033B603B68002297
:10052C000821144800F0C6FC4FF48073FB600223D2
:10053C003B6100237B610023BB610023FB6107F15E
:10054C000C0319464FF0904000F042FB0823FB606F
:10055C0001233B6100237B610023BB6107F10C038A
:10056C001946044800F034FB00BF2037BD4680BD5F
:10057C00001002400004004880B500AF00F0AFF955
:10058C0000F010F8FFF79CFF00F0FCF8082104487D
:10059C0000F0A8FC4FF4FA7000F012FAF6E700BF76
:1005AC000004004880B5A4B000AF07F14C0344220E
:1005BC000021184602F0A6F907F1380300221A6050
:1005CC005A609A60DA601A613B1D34220021184689
:1005DC0002F098F94FF4007000F0ACFC0346002BCD
:1005EC0001D000F040F80223FB644FF48073BB652C
:1005FC001023FB650023BB6707F14C03184600F082
:10060C00EFFC0346002B01D000F02DF80F23BB6349
:10061C000123FB6300233B6400237B640023BB6446
:10062C0007F138030021184601F01AF90346002B94
:10063C0001D000F018F802237B600023FB603B1D07
:10064C00184601F045FB0346002B01D000F00BF8D7
:10065C004FF080424FF08071002001F0E3F900BFB1
:10066C009037BD4680BD80B400AF00BFBD465DF87D
:10067C00047B704780B483B000AF0F4B1B6E0E4AE7
:10068C0043F0010313660C4B1B6E03F001037B60FC
:10069C007B68094B9B6D084A43F080539365064B6E
:1006AC009B6D03F080533B603B6800BF0C37BD462D
:1006BC005DF8047B704700BF0010024080B400AFAF
:1006CC0000BFBD465DF8047B704780B400AFFEE709
:1006DC0080B400AFFEE780B400AFFEE780B400AF9B
:1006EC00FEE780B400AF00BFBD465DF8047B7047E9
:1006FC0080B400AF00BFBD465DF8047B704780B48A
:10070C0000AF00BFBD465DF8047B704780B500AFFD
:10071C0000F038F900BF80BD80B400AF174BD3F8A0
:10072C008830164A43F47003C2F88830144B1B68A7
:10073C00134A43F001031360114B00229A60104BD3
:10074C001B680F4A23F0A85323F4102313600C4B9F
:10075C004FF48052DA600A4B1B68094A23F4802359
:10076C001360074B00229A61044B4FF000629A60B1
:10077C0000BFBD465DF8047B704700BF00ED00E094
:10078C000010024080B500AF144B154A1A60134B91
:10079C004FF4E1325A60114B00229A600F4B002249
:1007AC00DA600E4B00221A610C4B0C225A610B4B77
:1007BC0000229A61094B0022DA61084B00221A626E
:1007CC00064B00225A62054801F008FC0346002B38
:1007DC0001D0FFF748FF00BF80BD00BF28000020FC
:1007EC000044004080B58AB000AF786007F1140374
:1007FC0000221A605A609A60DA601A617B681B6882
:10080C00204A93423AD1204B9B6D1F4A43F400334C
:10081C0093651D4B9B6D03F400333B613B691A4B95
:10082C00DB6C194A43F00103D364174BDB6C03F008
:10083C000103FB60FB6804237B610223BB61002383
:10084C00FB6103233B6207237B6207F11403194608
:10085C004FF0904000F0BCF94FF400437B61022351
:10086C00BB610023FB6103233B6203237B6207F123
:10087C00140319464FF0904000F0AAF900BF283736
:10088C00BD4680BD0044004000100240DFF834D06B
:10089C00002103E00C4B5B58435004310B480C4BCC
:1008AC0042189A42F6D30B4A02E0002342F8043B6A
:1008BC00094B9A42F9D3FFF72FFF01F0FFFFFFF727
:1008CC005BFEFEE700A0002090290008000000203D
:1008DC000C0000200C000020AC000020FEE780B5CE
:1008EC0082B000AF0023FB71032000F03DF9002023
:1008FC0000F00EF80346002B02D00123FB7101E03F
:10090C00FFF7B8FEFB7918460837BD4680BD0000DE
:10091C0080B584B000AF78600023FB73164B1B6866
:10092C00002B22D0154B1A68134B1B684FF47A71AD
:10093C00B1FBF3F3B2FBF3F3184600F03CF90346BA
:10094C00002B0FD17B680F2B09D8002279684FF050
:10095C00FF3000F014F90A4A7B68136007E00123AA
:10096C00FB7304E00123FB7301E00123FB73FB7BAE
:10097C0018461037BD4680BD08000020000000203E
:10098C000400002080B400AF054B1A68054B1B68AF
:10099C001344034A136000BFBD465DF8047B7047E7
:1009AC00A80000200800002080B400AF034B1B6897
:1009BC001846BD465DF8047B704700BFA8000020B8
:1009CC0080B584B000AF7860FFF7EEFFB8607B684D
:1009DC00FB60FB68B3F1FF3F04D0094B1B68FA685E
:1009EC001344FB6000BFFFF7DFFF0246BB68D31A5E
:1009FC00FA689A42F7D800BF1037BD4680BD00BFD9
:100A0C000800002080B485B000AF78607B6803F0EC
:100A1C000703FB600C4BDB68BB60BA684FF6FF0347
:100A2C001340BB60FB681A02BB68134343F0BF63FF
:100A3C0043F40033BB60044ABB68D36000BF143777
:100A4C00BD465DF8047B704700ED00E080B400AF5C
:100A5C00044BDB681B0A03F007031846BD465DF820
:100A6C00047B704700ED00E080B483B000AF034618
:100A7C003960FB7197F90730002B0ADB3B68DAB25F
:100A8C000C4997F907301201D2B20B4483F80023BA
:100A9C000AE03B68DAB20849FB7903F00F03043B28
:100AAC001201D2B20B441A7600BF0C37BD465DF86A
:100ABC00047B704700E100E000ED00E080B489B0F9
:100ACC0000AFF860B9607A60FB6803F00703FB6164
:100ADC00FB69C3F10703042B28BF0423BB61FB692B
:100AEC000433062B02D9FB69033B00E000237B6136
:100AFC004FF0FF32BB6902FA03F3DA43BB681A40CA
:100B0C007B699A404FF0FF317B6901FA03F3D943BB
:100B1C007B680B40134318462437BD465DF8047BB5
:100B2C007047000080B582B000AF78607B68013BF5
:100B3C00B3F1807F01D301230FE00A4A7B68013BAC
:100B4C0053600F214FF0FF30FFF78EFF054B002253
:100B5C009A60044B07221A60002318460837BD46DA
:100B6C0080BD00BF10E000E080B582B000AF7860BF
:100B7C007868FFF747FF00BF0837BD4680BD80B5DA
:100B8C0086B000AF0346B9607A60FB7300237B61CB
:100B9C00FFF75CFF78617A68B9687869FFF78EFFB8
:100BAC00024697F90F3011461846FFF75DFF00BF5C
:100BBC001837BD4680BD80B582B000AF78607868CC
:100BCC00FFF7B0FF034618460837BD4680BD00004E
:100BDC0080B487B000AF7860396000237B614EE150
:100BEC003B681A6801217B6901FA03F31340FB602F
:100BFC00FB68002B00F040813B685B68022B03D044
:100C0C003B685B68122B23D17B69DA087B6808325E
:100C1C0053F822303B617B6903F007039B000F22E2
:100C2C0002FA03F3DB433A6913403B613B681A69F0
:100C3C007B6903F007039B0002FA03F33A69134341
:100C4C003B617B69DA087B680832396943F822100A
:100C5C007B681B683B617B695B00032202FA03F330
:100C6C00DB433A6913403B613B685B6803F003026A
:100C7C007B695B0002FA03F33A6913433B617B68BF
:100C8C003A691A603B685B68012B0BD03B685B6868
:100C9C00022B07D03B685B68112B03D03B685B6869
:100CAC00122B30D17B689B683B617B695B00032214
:100CBC0002FA03F3DB433A6913403B613B68DA68A1
:100CCC007B695B0002FA03F33A6913433B617B686F
:100CDC003A699A607B685B683B6101227B6902FA26
:100CEC0003F3DB433A6913403B613B685B681B09C8
:100CFC0003F001027B6902FA03F33A6913433B6187
:100D0C007B683A695A607B68DB683B617B695B0096
:100D1C00032202FA03F3DB433A6913403B613B685D
:100D2C009A687B695B0002FA03F33A6913433B61EF
:100D3C007B683A69DA603B685B6803F08053002B90
:100D4C0000F09A80554B1B6E544A43F00103136616
:100D5C00524B1B6E03F00103BB60BB68504A7B69AE
:100D6C009B08023352F823303B617B6903F0030389
:100D7C009B000F2202FA03F3DB433A6913403B61F9
:100D8C007B68B3F1904F13D07B68464A93420DD0E9
:100D9C007B68454A934207D07B68444A934201D111
:100DAC00032306E0072304E0022302E0012300E012
:100DBC0000237A6902F00302920093403A691343CC
:100DCC003B6137497B699B0802333A6941F8232020
:100DDC00374B1B683B61FB68DB433A6913403B6153
:100DEC003B685B6803F48033002B03D03A69FB68E3
:100DFC0013433B612E4A3B6913602D4B5B683B618F
:100E0C00FB68DB433A6913403B613B685B6803F466
:100E1C000033002B03D03A69FB6813433B61244A2F
:100E2C003B695360224B9B683B61FB68DB433A692F
:100E3C0013403B613B685B6803F48013002B03D0C9
:100E4C003A69FB6813433B61194A3B699360184B41
:100E5C00DB683B61FB68DB433A6913403B613B68F1
:100E6C005B6803F40013002B03D03A69FB6813434F
:100E7C003B610F4A3B69D3607B6901337B613B6803
:100E8C001A687B6922FA03F3002B7FF4A9AE00BF2A
:100E9C001C37BD465DF8047B704700BF0010024054
:100EAC00000001400004004800080048000C004805
:100EBC000004014080B483B000AF78600B467B80A7
:100ECC0013467B707B78002B03D07A887B689A6101
:100EDC0002E07A887B689A6200BF0C37BD465DF8E9
:100EEC00047B704780B483B000AF78600B467B8086
:100EFC007B685A697B881340002B03D07A887B6807
:100F0C009A6202E07A887B689A6100BF0C37BD4612
:100F1C005DF8047B7047000080B400AF044B1B6885
:100F2C0003F4C0631846BD465DF8047B704700BFF0
:100F3C000070004080B485B000AF78607B68B3F57A
:100F4C00007F30D1234B1B6803F4C063B3F5007FE3
:100F5C0038D0204B1B6823F4C0631E4A43F4007343
:100F6C0013601D4B1B68322202FB03F31B4AA2FBCE
:100F7C0003239B0C0133FB6002E0FB68013BFB602D
:100F8C00144B5B6903F48063B3F5806F02D1FB688B
:100F9C00002BF2D10F4B5B6903F48063B3F5806FC8
:100FAC0010D103230FE00B4B1B6803F4C063B3F5A4
:100FBC00806F07D0074B1B6823F4C063054A43F4CA
:100FCC0080631360002318461437BD465DF8047B1C
:100FDC00704700BF007000400000002083DE1B4300
:100FEC0080B58AB000AF78607B68002B02D10123FA
:100FFC0000F030BCA44B9B6803F00C033B62A24B8B
:10100C00DB6803F00303FB617B681B6803F01003D0
:10101C00002B00F0E2803B6A002B07D03B6A0C2BC4
:10102C0040F08980FB69012B40F08580964B1B6852
:10103C0003F00203002B06D07B68DB69002B02D186
:10104C00012300F007BC7B685A6A8F4B1B6803F0C6
:10105C000803002B04D08C4B1B6803F0F00305E055
:10106C00894BD3F894301B0903F0F003934223D23D
:10107C007B685B6A184600F0CBFD0346002B01D061
:10108C000123E7E3804B1B687F4A43F0080313609E
:10109C007D4B1B6823F0F0027B685B6A7A49134333
:1010AC000B60794B5B6823F47F427B681B6A1B02E5
:1010BC00754913434B6022E0734B1B68724A43F033
:1010CC0008031360704B1B6823F0F0027B685B6AAB
:1010DC006D4913430B606C4B5B6823F47F427B6858
:1010EC001B6A1B02684913434B607B685B6A18469A
:1010FC0000F08EFD0346002B01D00123AAE300F083
:10110C00C5FC0146604B9B681B0903F00F035F4A4B
:10111C00D35C03F01F0321FA03F35D4A13605D4BAC
:10112C001B681846FFF7F4FB0346FB75FB7D002B91
:10113C0052D0FB7D8EE37B68DB69002B32D0524BA7
:10114C001B68514A43F001031360FFF72DFCB86193
:10115C0008E0FFF729FC0246BB69D31A022B01D920
:10116C00032377E3484B1B6803F00203002BF0D0FA
:10117C00454B1B68444A43F008031360424B1B6801
:10118C0023F0F0027B685B6A3F4913430B603E4BD4
:10119C005B6823F47F427B681B6A1B023A4913434A
:1011AC004B601AE0384B1B68374A23F0010313607D
:1011BC00FFF7FAFBB86108E0FFF7F6FB0246BB69E4
:1011CC00D31A022B01D9032344E32F4B1B6803F0E2
:1011DC000203002BF0D100E000BF7B681B6803F01A
:1011EC000103002B74D03B6A082B05D03B6A0C2BF7
:1011FC000ED1FB69032B0BD1234B1B6803F400337B
:10120C00002B64D07B685B68002B60D1012321E349
:10121C007B685B68B3F5803F06D11B4B1B681A4A91
:10122C0043F4803313601DE07B685B68B3F5A02F3B
:10123C000CD1154B1B68144A43F480231360124BDA
:10124C001B68114A43F4803313600BE00E4B1B6890
:10125C000D4A23F4803313600B4B1B680A4A23F4AA
:10126C00802313607B685B68002B1CD0FFF79CFB12
:10127C00B86111E0FFF798FB0246BB69D31A642BE7
:10128C000AD90323E6E200BF001002403829000807
:10129C000000002004000020A04B1B6803F4003366
:1012AC00002BE7D014E0FFF77FFBB86108E0FFF7F5
:1012BC007BFB0246BB69D31A642B01D90323C9E219
:1012CC00964B1B6803F40033002BF0D100E000BFF9
:1012DC007B681B6803F00203002B60D03B6A042B75
:1012EC0005D03B6A0C2B19D1FB69022B16D18B4B09
:1012FC001B6803F48063002B05D07B68DB68002B34
:10130C0001D10123A6E2854B5B6823F0FE427B688A
:10131C001B691B06814913434B6040E07B68DB680B
:10132C00002B23D07D4B1B687C4A43F480731360E5
:10133C00FFF73AFBB86108E0FFF736FB0246BB69E2
:10134C00D31A022B01D9032384E2744B1B6803F4D8
:10135C008063002BF0D0714B5B6823F0FE427B68FE
:10136C001B691B066D4913434B6018E06B4B1B68E4
:10137C006A4A23F480731360FFF716FBB86108E028
:10138C00FFF712FB0246BB69D31A022B01D90323C8
:10139C0060E2624B1B6803F48063002BF0D17B6826
:1013AC001B6803F00803002B7FD07B685B69002B64
:1013BC005FD05A4BD3F894303B617B689A693B6998
:1013CC0003F010039A4237D03B6903F00203002B61
:1013DC0006D03B6903F00103002B01D1012339E254
:1013EC003B6903F00103002B1BD04C4BD3F894301A
:1013FC004A4A23F00103C2F89430FFF7D5FAB861DA
:10140C0008E0FFF7D1FA0246BB69D31A112B01D9B8
:10141C0003231FE2414BD3F8943003F00203002B5B
:10142C00EFD13E4BD3F8943023F010027B689B69CC
:10143C003A491343C1F89430384BD3F89430374AB7
:10144C0043F00103C2F89430FFF7AEFAB86108E03C
:10145C00FFF7AAFA0246BB69D31A112B01D9032351
:10146C00F8E12E4BD3F8943003F00203002BEFD0AD
:10147C001BE02A4BD3F89430284A23F00103C2F81E
:10148C009430FFF791FAB86108E0FFF78DFA024645
:10149C00BB69D31A112B01D90323DBE11F4BD3F802
:1014AC00943003F00203002BEFD17B681B6803F030
:1014BC000403002B00F0C280002387F82730174B61
:1014CC009B6D03F08053002B0ED1144B9B6D134A74
:1014DC0043F080539365114B9B6D03F08053FB607D
:1014EC00FB68012387F827300D4B1B6803F48073CE
:1014FC00002B1DD10A4B1B68094A43F480731360FF
:10150C00FFF752FAB8610DE0FFF74EFA0246BB69DD
:10151C00D31A022B06D903239CE100BF0010024012
:10152C0000700040AF4B1B6803F48073002BEBD0B2
:10153C007B689B6803F00103002B2CD0AA4BD3F8DB
:10154C00903023F080027B689B6803F08003A649EF
:10155C001343C1F890307B689B6803F00403002BA5
:10156C0010D0A14BD3F890309F4A43F00403C2F83B
:10157C0090309D4BD3F890309B4A43F00103C2F856
:10158C00903018E0984BD3F89030974A43F0010311
:10159C00C2F890300FE0944BD3F89030924A23F07D
:1015AC000103C2F89030904BD3F890308E4A23F060
:1015BC000403C2F890307B689B68002B16D0FFF7B1
:1015CC00F3F9B8610AE0FFF7EFF90246BB69D31AE9
:1015DC0041F28832934201D903233BE1824BD3F889
:1015EC00903003F00203002BEDD01DE0FFF7DCF987
:1015FC00B8610AE0FFF7D8F90246BB69D31A41F289
:10160C008832934201D9032324E1774BD3F89030ED
:10161C0003F00203002BEDD1734BD3F89030724AD8
:10162C0023F08003C2F8903097F82730012B05D1B6
:10163C006D4B9B6D6C4A23F0805393657B681B68E4
:10164C0003F02003002B3CD07B689B6A002B1CD042
:10165C00654BD3F89830644A43F00103C2F89830D4
:10166C00FFF7A2F9B86108E0FFF79EF90246BB69E3
:10167C00D31A022B01D90323ECE05B4BD3F898303F
:10168C0003F00203002BEFD01BE0574BD3F898303C
:10169C00554A23F00103C2F89830FFF785F9B86179
:1016AC0008E0FFF781F90246BB69D31A022B01D976
:1016BC000323CFE04C4BD3F8983003F00203002BFC
:1016CC00EFD17B68DB6A002B00F0C3803B6A0C2BEC
:1016DC0000F081807B68DB6A022B56D1424B1B6881
:1016EC00414A23F080731360FFF75EF9B86108E09C
:1016FC00FFF75AF90246BB69D31A022B01D903230F
:10170C00A8E0394B1B6803F00073002BF0D1364B6B
:10171C00DA68364B13407A68116B7A68526B013A6F
:10172C00120111437A68926B120211437A68D26BE0
:10173C005208013A520511437A68126C5208013A68
:10174C0052060A4328491343CB60274B1B68264A91
:10175C0043F080731360244BDB68234A43F080739F
:10176C00D360FFF721F9B86108E0FFF71DF90246D5
:10177C00BB69D31A022B01D903236BE01A4B1B68EC
:10178C0003F00073002BF0D063E0174B1B68164A74
:10179C0023F080731360144BDB68134A23F00303AC
:1017AC00D360114BDB68104A23F08873D360FFF7CA
:1017BC00FBF8B86108E0FFF7F7F80246BB69D31AEB
:1017CC00022B01D9032345E0074B1B6803F0007380
:1017DC00002BF0D13DE07B68DB6A012B08D10123A3
:1017EC0038E000BF00700040001002408C809FF970
:1017FC001A4BDB68FB61FB6903F003027B681B6B14
:10180C009A4224D1FB6903F070027B685B6B013B4D
:10181C001B019A421BD1FB6903F4FE427B689B6B54
:10182C001B029A4213D1FB6903F4C0027B68DB6B89
:10183C005B08013B5B059A4209D1FB6903F0C0626E
:10184C007B681B6C5B08013B5B069A4201D0012351
:10185C0000E0002318462837BD4680BD001002402A
:10186C0080B584B000AF786039607B68002B01D103
:10187C000123C8E0664B1B6803F007033A689A42E1
:10188C0010D9634B1B6823F0070261493B68134373
:10189C000B605F4B1B6803F007033A689A4201D058
:1018AC000123B0E07B681B6803F00103002B4CD0D4
:1018BC007B685B68032B07D1564B1B6803F00073E6
:1018CC00002B21D101239EE07B685B68022B07D1A2
:1018DC00504B1B6803F40033002B15D1012392E00D
:1018EC007B685B68002B07D14A4B1B6803F0020333
:1018FC00002B09D1012386E0464B1B6803F480635F
:10190C00002B01D101237EE0424B9B6823F00302A4
:10191C007B685B683F4913438B60FFF745F8F860C1
:10192C000AE0FFF741F80246FB68D31A41F288320D
:10193C00934201D9032366E0364B9B6803F00C02FB
:10194C007B685B689B009A42EBD17B681B6803F059
:10195C000203002B08D02F4B9B6823F0F0027B680E
:10196C009B682C4913438B60294B1B6803F00703BE
:10197C003A689A4210D2264B1B6823F0070224497E
:10198C003B6813430B60224B1B6803F007033A6858
:10199C009A4201D0012336E07B681B6803F00403F4
:1019AC00002B08D01B4B9B6823F4E0627B68DB6840
:1019BC00184913438B607B681B6803F00803002BEA
:1019CC0009D0144B9B6823F460527B681B69DB00C5
:1019DC00104913438B6000F059F801460D4B9B687E
:1019EC001B0903F00F030C4AD35C03F01F0321FA0D
:1019FC0003F30A4A13600A4B1B681846FEF788FF6C
:101A0C000346FB72FB7A18461037BD4680BD00BFFB
:101A1C00002002400010024038290008000000207D
:101A2C000400002080B58AB000AFF860B9607A601D
:101A3C00154BDB6C144A43F00103D364124BDB6C83
:101A4C0003F001033B613B694FF480737B6102231C
:101A5C00BB6102233B620023FB6100237B6207F125
:101A6C00140319464FF09040FFF7B2F8064B9B68F1
:101A7C0023F0FE42B9687B680B43034913438B6028
:101A8C0000BF2837BD4680BD0010024080B489B02D
:101A9C0000AF0023FB610023BB613D4B9B6803F04F
:101AAC000C033B613A4BDB6803F00303FB603B69BF
:101ABC00002B05D03B690C2B21D1FB68012B1ED1CF
:101ACC00334B1B6803F00803002B07D1304BD3F8C2
:101ADC0094301B0A03F00F03FB6105E02C4B1B68D1
:101AEC001B0903F00F03FB612A4AFB6952F82330F0
:101AFC00FB613B69002B0DD1FB69BB610AE03B69C3
:101B0C00042B02D1244BBB6104E03B69082B01D1AF
:101B1C00224BBB613B690C2B33D11D4BDB6803F0B3
:101B2C000303BB60BB68022B02D0032B03D005E080
:101B3C00194B7B6105E0194B7B6102E0FB697B6112
:101B4C0000BF134BDB681B0903F0070301337B60F9
:101B5C000F4BDB681B0A03F07F037A6902FB03F26D
:101B6C007B68B2FBF3F37B61094BDB685B0E03F024
:101B7C00030301335B003B607A693B68B2FBF3F310
:101B8C00BB61BB6918462437BD465DF8047B7047C2
:101B9C0000100240502900080024F40000127A00C2
:101BAC0080B400AF034B1B681846BD465DF8047B40
:101BBC00704700BF0000002080B500AFFFF7F0FFBA
:101BCC000146064B9B681B0A03F00703044AD35CCF
:101BDC0003F01F0321FA03F3184680BD00100240E6
:101BEC004829000880B500AFFFF7DAFF0146064B25
:101BFC009B68DB0A03F00703044AD35C03F01F0362
:101C0C0021FA03F3184680BD001002404829000851
:101C1C0080B586B000AF786000233B612A4B9B6D8A
:101C2C0003F08053002B03D0FFF776F9786114E0B2
:101C3C00254B9B6D244A43F080539365224B9B6D3F
:101C4C0003F08053FB60FB68FFF766F978611E4B6D
:101C5C009B6D1D4A23F0805393657B69B3F5007F20
:101C6C000BD17B68802B19D97B68A02B02D902235E
:101C7C003B6113E001233B6110E07B68802B02D9B0
:101C8C0003233B610AE07B68802B02D102233B617A
:101C9C0004E07B68702B01D101233B610B4B1B686B
:101CAC0023F0070209493B6913430B60074B1B6880
:101CBC0003F007033A699A4201D0012300E00023A4
:101CCC0018461837BD4680BD001002400020024067
:101CDC0080B586B000AF78600023FB740023BB7422
:101CEC007B681B6803F40033002B00F09E800023FC
:101CFC007B74464B9B6D03F08053002B01D1012369
:101D0C0000E00023002B0DD0404B9B6D3F4A43F06D
:101D1C00805393653D4B9B6D03F08053BB60BB6858
:101D2C0001237B743A4B1B68394A43F4807313606C
:101D3C00FEF73AFEF86009E0FEF736FE0246FB6855
:101D4C00D31A022B02D90323FB7405E0304B1B681A
:101D5C0003F48073002BEFD0FB7C002B5AD12B4B60
:101D6C00D3F8903003F440737B617B69002B1ED059
:101D7C007B681B6B7A699A4219D0244BD3F890304C
:101D8C0023F440737B61214BD3F890301F4A43F40A
:101D9C008033C2F890301D4BD3F890301B4A23F49B
:101DAC008033C2F89030194A7B69C2F890307B6955
:101DBC0003F00103002B16D0FEF7F6FDF8600BE0E4
:101DCC00FEF7F2FD0246FB68D31A41F288329342C9
:101DDC0002D90323FB7406E00C4BD3F8903003F0CC
:101DEC000203002BECD0FB7C002B0BD1074BD3F860
:101DFC00903023F440727B681B6B04491343C1F889
:101E0C00903009E0FB7CBB7406E000BF0010024080
:101E1C0000700040FB7CBB747B7C012B05D16E4BAE
:101E2C009B6D6D4A23F0805393657B681B6803F0B0
:101E3C000103002B0AD0684BD3F8883023F003023F
:101E4C007B685B6864491343C1F888307B681B6806
:101E5C0003F00203002B0AD05F4BD3F8883023F039
:101E6C000C027B689B685C491343C1F888307B6823
:101E7C001B6803F00403002B0AD0574BD3F88830AF
:101E8C0023F030027B68DB6853491343C1F8883078
:101E9C007B681B6803F02003002B0AD04E4BD3F851
:101EAC00883023F440627B681B694B491343C1F8AB
:101EBC0088307B681B6803F40073002B0AD0464BF8
:101ECC00D3F8883023F440227B681B6A42491343C1
:101EDC00C1F888307B681B6803F48063002B0AD040
:101EEC003D4BD3F8883023F440127B685B6A3A4947
:101EFC001343C1F888307B681B6803F04003002B48
:101F0C000AD0354BD3F8883023F440527B685B6998
:101F1C0031491343C1F888307B681B6803F0800398
:101F2C00002B0AD02C4BD3F8883023F440427B682A
:101F3C009B6929491343C1F888307B681B6803F4FB
:101F4C008073002B0AD0244BD3F8883023F4403212
:101F5C007B68DB6920491343C1F888307B681B68B8
:101F6C0003F40053002B15D01B4BD3F8883023F00F
:101F7C0040627B689B6A18491343C1F888307B68C0
:101F8C009B6AB3F1006F05D1134BDB68124A43F423
:101F9C008013D3607B681B6803F48023002B15D05F
:101FAC000D4BD3F8883023F040627B68DB6A0A491A
:101FBC001343C1F888307B68DB6AB3F1006F05D13D
:101FCC00054BDB68044A43F48013D360BB7C184692
:101FDC001837BD4680BD00BF0010024080B582B0EE
:101FEC0000AF78607B68002B01D1012340E07B6857
:101FFC005B6F002B06D17B68002283F87020786819
:10200C00FEF7F0FB7B6824225A677B681B681A6812
:10201C007B681B6822F001021A60786800F02CF8CB
:10202C000346012B01D1012322E07B685B6A002B64
:10203C0002D0786800F012FB7B681B685A687B68DA
:10204C001B6822F490425A607B681B689A687B6814
:10205C001B6822F02A029A607B681B681A687B68EE
:10206C001B6842F001021A60786800F099FB034685
:10207C0018460837BD4680BD2DE9904888B000AFA2
:10208C00786000237B610023FB740023FB607B687A
:10209C009A687B681B691A437B685B691A437B6887
:1020AC00DB691343FB617B681B681A68AF4B1340F9
:1020BC007A681268F9690B4313607B681B685B686C
:1020CC0023F440517B68DA687B681B680A435A60CA
:1020DC007B689B69FB617B681B68A54A934204D0B3
:1020EC007B681B6AFA691343FB617B681B689B68FE
:1020FC0023F430617B681B68FA690A439A607B6839
:10210C001B689C4A934221D19B4BD3F8883003F037
:10211C000303032B16D801A252F823F0392100082F
:10212C00452100083F2100084B2100080123FB76C4
:10213C0098E00223FB7695E00423FB7692E00823DB
:10214C00FB768FE01023FB7600BF8BE07B681B686F
:10215C008A4A934234D1884BD3F8883003F00C036D
:10216C000C2B29D801A252F823F000BFAD21000896
:10217C00C5210008C5210008C5210008B9210008A7
:10218C00C5210008C5210008C5210008B32100089D
:10219C00C5210008C5210008C5210008BF21000881
:1021AC000023FB765EE00223FB765BE00423FB76E8
:1021BC0058E00823FB7655E01023FB7600BF51E076
:1021CC007B681B686E4A934220D16B4BD3F88830E6
:1021DC0003F03003102B0FD0102B02D8002B05D09E
:1021EC0010E0202B05D0302B09D00BE00023FB7620
:1021FC0038E00223FB7635E00423FB7632E008233B
:10220C00FB762FE01023FB7600BF2BE07B681B686E
:10221C00574A934224D1584BD3F8883003F4406387
:10222C00B3F5806F12D0B3F5806F02D8002B07D0B6
:10223C0012E0B3F5006F06D0B3F5406F09D00BE098
:10224C000023FB760EE00223FB760BE00423FB76E7
:10225C0008E00823FB7605E01023FB7600BF01E0C5
:10226C001023FB767B681B68414A934240F0F48054
:10227C00FB7E082B23D801A252F823F0AD220008D4
:10228C00CB220008B5220008CB220008BB22000894
:10229C00CB220008CB220008CB220008C322000866
:1022AC00FFF78AFCF8600DE0364BFB600AE0FFF7A5
:1022BC00EDFBF86006E04FF40043FB6002E0012305
:1022CC00FB7400BFFB68002B00F0B9817B685A6877
:1022DC0013465B001344FA689A4205D37B685B682B
:1022EC001B03FA689A4202D90123FB74A7E1FB7E17
:1022FC00082B00F29E8001A252F823F02D23000837
:10230C003F240008952300083F240008C923000837
:10231C003F2400083F2400083F240008152400082F
:10232C00FFF74AFC034619464FF000024FF000033A
:10233C004FF00004140244EA11640B027A685268EC
:10234C00520811464FF0000213EB010B44EB020C48
:10235C00584661467B685B684FF000041A4623467A
:10236C00FDF72EFF03460C467B6165E0F369FFEF3A
:10237C000080004000380140001002400044004042
:10238C00004800400024F4007B685B685B084FF059
:10239C000004B1494FF0000213EB010B44EB020CAB
:1023AC00584661467B685B684FF000041A4623462A
:1023BC00FDF706FF03460C467B613DE0FFF766FB2D
:1023CC00034619464FF000024FF000034FF0000493
:1023DC00140244EA11640B027A68526852081146DE
:1023EC004FF0000213EB010B44EB020C5846614614
:1023FC007B685B684FF000041A462346FDF7E0FE4D
:10240C0003460C467B6117E07B685B685B084FF00A
:10241C00000413F5000044F100017B685B684FF089
:10242C0000041A462346FDF7CBFE03460C467B619F
:10243C0002E00123FB7400BF7B69B3F5407F08D336
:10244C007B69B3F5801F04D27B681B687A69DA60FC
:10245C00F5E00123FB74F2E07B68DB69B3F5004F18
:10246C007FD1FB7E082B5CD801A252F823F000BF71
:10247C00A1240008BF240008DD2400082F25000833
:10248C00F92400082F2500082F2500082F25000807
:10249C0017250008FFF790FB03465A007B685B6822
:1024AC005B081A447B685B68B2FBF3F39BB27B61FD
:1024BC003AE0FFF797FB03465A007B685B685B08C2
:1024CC001A447B685B68B2FBF3F39BB27B612BE035
:1024DC007B685B685B0803F1F47303F590437A68DF
:1024EC005268B3FBF2F39BB27B611DE0FFF7CEFAAF
:1024FC0003465A007B685B685B081A447B685B6820
:10250C00B2FBF3F39BB27B610EE07B685B685B080C
:10251C0003F580327B685B68B2FBF3F39BB27B61A3
:10252C0002E00123FB7400BF7B690F2B16D97B697A
:10253C00B3F5803F12D27B699BB223F00F037B81F2
:10254C007B695B089BB203F007039AB27B89134348
:10255C007B817B681B687A89DA6070E00123FB74ED
:10256C006DE0FB7E082B59D801A252F823F000BF76
:10257C00A1250008BD250008D9250008292600083A
:10258C00F525000829260008292600082926000818
:10259C0011260008FFF710FB02467B685B685B089E
:1025AC001A447B685B68B2FBF3F39BB27B6138E047
:1025BC00FFF718FB02467B685B685B081A447B6874
:1025CC005B68B2FBF3F39BB27B612AE07B685B68D0
:1025DC005B0803F5740303F510537A685268B3FB78
:1025EC00F2F39BB27B611CE0FFF750FA02467B686A
:1025FC005B685B081A447B685B68B2FBF3F39BB2C5
:10260C007B610EE07B685B685B0803F500427B68CE
:10261C005B68B2FBF3F39BB27B6102E00123FB74BA
:10262C0000BF7B690F2B08D97B69B3F5803F04D2BF
:10263C007B681B687A69DA6001E00123FB747B68B4
:10264C0000221A667B6800225A66FB7C18462037EB
:10265C00BD46BDE8908800BF000024F480B483B070
:10266C0000AF78607B685B6A03F00103002B0AD033
:10267C007B681B685B6823F400317B689A6A7B6813
:10268C001B680A435A607B685B6A03F00203002BE9
:10269C000AD07B681B685B6823F480317B68DA6A3C
:1026AC007B681B680A435A607B685B6A03F004030F
:1026BC00002B0AD07B681B685B6823F480217B6845
:1026CC001A6B7B681B680A435A607B685B6A03F071
:1026DC000803002B0AD07B681B685B6823F400415D
:1026EC007B685A6B7B681B680A435A607B685B6A21
:1026FC0003F01003002B0AD07B681B689B6823F443
:10270C0080517B689A6B7B681B680A439A607B6874
:10271C005B6A03F02003002B0AD07B681B689B6864
:10272C0023F400517B68DA6B7B681B680A439A6060
:10273C007B685B6A03F04003002B1AD07B681B6834
:10274C005B6823F480117B681A6C7B681B680A43F6
:10275C005A607B681B6CB3F5801F0AD17B681B68C1
:10276C005B6823F4C0017B685A6C7B681B680A4366
:10277C005A607B685B6A03F08003002B0AD07B688D
:10278C001B685B6823F400217B689A6C7B681B6870
:10279C000A435A6000BF0C37BD465DF8047B704796
:1027AC0080B586B002AF78607B680022DA67FEF7EE
:1027BC00FBF8F8607B681B681B6803F00803082BA8
:1027CC000ED16FF07E430093FB6800224FF4001192
:1027DC00786800F02AF80346002B01D0032320E090
:1027EC007B681B681B6803F00403042B0ED16FF08D
:1027FC007E430093FB6800224FF48001786800F060
:10280C0014F80346002B01D003230AE07B68202236
:10281C005A677B6820229A677B68002283F87020B5
:10282C00002318461037BD4680BD80B584B000AF7C
:10283C00F860B9603B601346FB712AE0BB69B3F1E9
:10284C00FF3F26D0FEF7B0F802463B68D31ABA69B0
:10285C009A4202D3BB69002B1BD1FB681B681A6818
:10286C00FB681B6822F4D0721A60FB681B689A68BC
:10287C00FB681B6822F001029A60FB6820225A67F1
:10288C00FB6820229A67FB68002283F870200323E0
:10289C000FE0FB681B68DA69BB681340BA689A42A0
:1028AC000CBF01230023DBB21A46FB799A42C5D038
:1028BC00002318461037BD4680BD000070B50D4E84
:1028CC000D4CA41BA4100025A54209D10B4E0C4C99
:1028DC0000F020F8A41BA4100025A54205D170BD62
:1028EC0056F8253098470135EEE756F825309847CD
:1028FC000135F2E788290008882900088829000892
:10290C008C29000802440346934200D1704703F817
:10291C00011BF9E7F8B500BFF8BC08BC9E46704730
:0C292C00F8B500BFF8BC08BC9E46704720
:102938000000000000000000010203040607080967
:102948000000000001020304A0860100400D0300FE
:10295800801A060000350C0040420F0080841E00DB
:1029680000093D0000127A000024F40000366E01D0
:082978000048E801006CDC02DC
:082980007CD8FF7F010000007C
:04298800B101000891
:04298C008D010008B1
:0C29900000093D001000000001000000E4
:04000005080008994E
:00000001FF
